:020000040000FA
:04000000D1303A2899
:08000800A000030EA100831209
:100010008B1C32288B1031181428B11C3228643004
:10002000010203183128182800001628172818285C
:1000300019281A281B281C281D281E281F283110A3
:10004000B114A810031005190314AA0DA90DA80DC9
:10005000B00B322831152A08AF002908AE00280855
:10006000AD00B11081010B11210E8300A00E200EF6
:02007000090085
:0C007400203084008001840A80300402E7
:10008000031C3C281230B000082283160C30850572
:1000900087018312850187010730990000309A009B
:1000A000103083168E008312603083168F00831207
:1000B0000030831691009F008312C83083168100A0
:1000C000831231309000003083168C008312103080
:1000D0008B00831600309B001C141A088312BC008E
:1000E000831610309B001C141A088312BD0083165F
:1000F00030309B001C141A088312DE006D2381012E
:100100008E018F010B118B100B108C018B17962019
:100110003119AC20B30B9428031085190314B90DC1
:10012000F030390203196421B023872864003118A4
:1001300008000B1D08000B11B11031141230B00073
:10014000051DA728321483160113831208003210EC
:10015000831601178312080031110130B7008B1389
:100160002030370783169B001C141A088312A40042
:10017000A500C030A5061030370783169B001C145D
:100180001A088312A3000030370783169B001C1443
:100190001A088312A2008B17321CD42822090339B3
:1001A000A200A309A409A50922082D02031D5E29A6
:1001B00023082E02031D5E2924082F02031D5E2939
:1001C00001303702031DE9283D18E9283D143E148B
:1001D000152202303702031DF228BD18F228BD1483
:1001E0003E14272203303702031DFB283D19FB284C
:1001F0003D153E14392204303702031D0429BD1970
:100200000429BD153E144B2205303702031D0D296C
:100210003D1A0D293D163E145D2206303702031D9E
:100220001629BD1A1629BD163E146E220730370254
:10023000031D1F293D1B1F293D173E147F22083037
:100240003702031D2829BD1B2829BD173E14902203
:1002500009303702031D31295E1831295E143E141E
:10026000A1220A303702031D3A29DE183A29DE148A
:100270003E14BA220B303702031D43295E1943296D
:100280005E153E14D3220C303702031D4C29DE19B3
:100290004C29DE153E14E8220D303702031D552986
:1002A0005E1A55295E163E14FD220E303702031DDC
:1002B0005E29DE1A5E29DE163E141223B70A0F30BD
:1002C000370203180800AF280130B600B300B400AD
:1002D000B500B70085018701B1139620B30BB4298F
:1002E000031085190314B90DF03039020319DB2905
:1002F000B40BB42901303702031927230230370227
:1003000003192C2303303702031931230430370239
:10031000031936230530370203193B230630370211
:1003200003194023073037020319452308303702E9
:1003300003194A230930370203194F230A303702C1
:10034000031954230B303702031959230C30370299
:1003500003195E230D303702031963230E30370271
:10036000031968239630B400311D6D293111321CF8
:10037000BE292D090339AD00AE09AF092F1CB113F9
:100380002F1C6D29B11B6D292E186D29B1178B13E8
:1003900020303707BB002F08BA00F3211030370791
:1003A000BB002E08BA00F32100303707BB002D0830
:1003B000BA00F3218B1785018701B70AB6010F3008
:1003C0003702031C6D296D2308003E1C08003E10F7
:1003D0001030BB003D08BA00F3213030BB005E088E
:1003E000BA00F32108008B133A0883161C159A00F3
:1003F00083123B0883169B0055309D00AA309D0058
:100400009C1464009C18012A1C1183128B1708008D
:10041000FF30C800CA15CB15CC15CD15CE15CF159C
:10042000D015D115D215D31508000130BD05003007
:10043000DE054030C405C0000030C200C6004030B8
:10044000C505C1000030C300C7005F1008000230BE
:10045000BD050030DE050830C405C0000030C20014
:10046000C6004030C505C1000030C300C7005F10A2
:1004700008000430BD050030DE050830C405C000AA
:100480000030C200C6004030C505C1004030C30086
:10049000C7005F1008000830BD050030DE05883059
:1004A000C405C0000030C200C6000030C505C10050
:1004B0000030C300C7005F1008001030BD050030D9
:1004C000DE058830C405C0008030C200C6000030A0
:1004D000C505C1000030C300C70008002030BD05BD
:1004E0000030DE051030C405C0000030C200C60078
:1004F0000030C505C1000030C300C700080040300F
:10050000BD050030DE052030C405C0000030C2004B
:10051000C6000030C505C1000030C300C700080098
:100520008030BD050030DE052030C405C00020301D
:10053000C200C6000030C505C1000030C300C700BE
:1005400008000030BD05C130DE0508304418013A0E
:10055000C418023AC405C00000304618013AC61853
:10056000023AC200C6008030C505C1000030C30099
:10057000C70008000030BD05C230DE050830441851
:10058000013AC418023AC405C00000304618013AC6
:10059000C618023AC200C6008030C505C1008030CE
:1005A000C300C70008000030BD05C430DE050A30B6
:1005B000C405C0000030C200C6000030C51B803A30
:1005C000C505C1000030C71B803AC300C700080042
:1005D0000030BD05C830DE050A30C405C000023059
:1005E000C200C6000030C51B803AC505C1000030FE
:1005F000C71B803AC300C70008000030BD05D030DB
:10060000DE050930C405C0000030C200C60000305D
:10061000C51B803AC505C1000030C71B803AC30026
:10062000C70008000030BD05E030DE050930C40514
:10063000C0000130C200C6000030C51B803AC505AD
:10064000C1000030C71B803AC300C700080000305B
:1006500085061130870608000230850610308706AF
:100660000800023085061030870608000230850633
:1006700020308706080002308506203087060800F3
:1006800000308506023087060800003085060430F9
:10069000870608000030850604308706080002300F
:1006A0008506083087060800023085060830870670
:1006B00008002230850600308706080022308506B3
:1006C00000308706080012308506003087060800D3
:1006D000123085060030870608003D181522BD1827
:1006E00027223D193922BD194B223D1A5D22BD1A20
:1006F0006E223D1B7F22BD1B90225E18A122DE18B8
:10070000BA225E19D322DE19E8225E1AFD22DE1A11
:1007100012230800B601B301B4013C1C922BBC01AA
:10072000BC14942BBC013C143C08B6006400982B0C
:10073000992B9A2B9B2B9C2BFF30B41B8500B41F4D
:100740008501B30B962BB40B962B0310B60CB60891
:10075000031D962B0030BB003C08BA00F3210800B3
:100760008F08031908008F0178308E00C80FDA2D2A
:10077000C80A441CE02B461CD12BCA1CC22BCA0140
:100780004A15EE2B4A1DC72BCA01CA15EE2BCA1DEE
:10079000CC2BCA014A16EE2B4A1EEE2BCA01CA14F4
:1007A000EE2B4A1DD62BCA014A16EE2BCA1DDB2B97
:1007B000CA014A16EE2B4A1EEE2BCA01CA14EE2BB2
:1007C000CA1CE52BCA014A15EE2B4A1DEA2BCA01A9
:1007D000CA15EE2B4A1EEE2BCA014A15C41C152C55
:1007E000C61C062CCB1CF72BCB014B15232C4B1D09
:1007F000FC2BCB01CB15232CCB1D012CCB014B1695
:10080000232C4B1E232CCB01CB14232C4B1D0B2C48
:10081000CB014B16232CCB1D102CCB014B16232CBC
:100820004B1E232CCB01CB14232CCB1C1A2CCB011D
:100830004B15232C4B1D1F2CCB01CB15232C4B1EF2
:10084000232CCB014B15441D4A2C461D3B2CCC1CA4
:100850002C2CCC014C15582C4C1D312CCC01CC151A
:10086000582CCC1D362CCC014C16582C4C1E582C18
:10087000CC01CC14582C4C1D402CCC014C16582CBF
:10088000CC1D452CCC014C16582C4C1E582CCC01A0
:10089000CC14582CCC1C4F2CCC014C15582C4C1D76
:1008A000542CCC01CC15582C4C1E582CCC014C157A
:1008B000C41D802CC61D712CCD1C622CCD014D1584
:1008C0005F138E2C4D1D672CCD01CD158E2CCD1DAB
:1008D0006C2CCD014D168E2C4D1E8E2CCD01CD14C1
:1008E0008E2C4D1D762CCD014D168E2CCD1D7B2CC6
:1008F000CD014D168E2C4D1E8E2CCD01CD148E2C7F
:10090000CD1C852CCD014D158E2C4D1D8A2CCD0175
:10091000CD158E2C4D1E8E2CCD014D155F1BB72C89
:10092000441EB72C461EA82CCE1C992CCE014E1569
:10093000C52C4E1D9E2CCE01CE15C52CCE1DA32C34
:10094000CE014E16C52C4E1EC52CCE01CE14C52C84
:100950004E1DAD2CCE014E16C52CCE1DB22CCE0197
:100960004E16C52C4E1EC52CCE01CE14C52CCE1C49
:10097000BC2CCE014E15C52C4E1DC12CCE01CE1562
:10098000C52C4E1EC52CCE014E15C41EEC2CC61E09
:10099000DD2CCF1CCE2CCF014F15FA2C4F1DD32CA4
:1009A000CF01CF15FA2CCF1DD82CCF014F16FA2C22
:1009B0004F1EFA2CCF01CF14FA2C4F1DE22CCF0181
:1009C0004F16FA2CCF1DE72CCF014F16FA2C4F1ED5
:1009D000FA2CCF01CF14FA2CCF1CF12CCF014F15DC
:1009E000FA2C4F1DF62CCF01CF15FA2C4F1EFA2CE6
:1009F000CF014F15441F212D461F122DD01C032D52
:100A0000D00150152F2D501D082DD001D0152F2DA0
:100A1000D01D0D2DD00150162F2D501E2F2DD00181
:100A2000D0142F2D501D172DD00150162F2DD01D55
:100A30001C2DD00150162F2D501E2F2DD001D0145B
:100A40002F2DD01C262DD00150152F2D501D2B2DB4
:100A5000D001D0152F2D501E2F2DD0015015C41FA1
:100A6000562DC61F472DD11C382DD1015115642D8F
:100A7000511D3D2DD101D115642DD11D422DD10126
:100A80005116642D511E642DD101D114642D511DB8
:100A90004C2DD1015116642DD11D512DD10151166E
:100AA000642D511E642DD101D114642DD11C5B2DF8
:100AB000D1015115642D511D602DD101D115642D29
:100AC000511E642DD1015115451F8C2D471F7D2DC1
:100AD000D21C6E2DD2015215DF139A2D521D732D8B
:100AE000D201D2159A2DD21D782DD20152169A2DEF
:100AF000521E9A2DD201D2149A2D521D822DD2014E
:100B000052169A2DD21D872DD20152169A2D521EA1
:100B10009A2DD201D2149A2DD21C912DD2015215A8
:100B20009A2D521D962DD201D2159A2D521E9A2D14
:100B3000D2015215DF1BC32DC51FC32DC71FB42DF6
:100B4000D31CA52DD3015315D12D531DAA2DD3018F
:100B5000D315D12DD31DAF2DD3015316D12D531E37
:100B6000D12DD301D314D12D531DB92DD30153163B
:100B7000D12DD31DBE2DD3015316D12D531ED12DF2
:100B8000D301D314D12DD31CC82DD3015315D12D8E
:100B9000531DCD2DD301D315D12D531ED12DD301EE
:100BA0005315E5214008C4004108C5005F18DF1453
:100BB0005F1CDF104808C9000C304A05031D0512F0
:100BC0000C304B05031D85120C304C05031D051020
:100BD0000C304D05031D85100C304E05031D87108C
:100BE0000C304F05031D07110C305005031D071075
:100BF0000C305105031D87120C305205031D0712DE
:100C00000C305305031D871149080E020318342EBA
:100C100012304A05031D051612304B05031D8516BB
:100C200012304C05031D051412304D05031D8514AB
:100C300012304E05031D871412304F05031D071592
:100C400012305005031D071412305105031D87167D
:100C500012305205031D071612305305031D871568
:100C6000FF304802031908008F08031D0800962072
:100C700049080E02031C342E18304A05031D0512C4
:100C800006304A05031D051618304B05031D851255
:100C900006304B05031D851618304C05031D051045
:100CA00006304C05031D051418304D05031D851035
:100CB00006304D05031D851418304E05031D8710A1
:100CC00006304E05031D871418304F05031D07110C
:100CD00006304F05031D071518305005031D07107A
:100CE00006305005031D071418305105031D8712E7
:100CF00006305105031D871618305205031D0712D3
:100D000006305205031D071618305305031D8711C1
:0A0D100006305305031D8715080087
:084000000900030004000500A3
:02400E00CC33B1
:10420000010003000300030003000200020002009B
:104210000200000000000000000003000300FF0097
:10422000020000000000000000000000000000008C
:104230000000C000C000C000C000C000C000FF00FF
:10424000FF00C300F300CF00FF00C300F300CF0066
:10425000FF00C300F300CF00FF00C300F300FF0026
:104260000100FF00FF00FF00FF00FF00FF00FF0054
:10427000FF00FF00FF00FF00FF00FF00FF00FF0046
:10428000FF00FF00FF00FF00FF00FF00FF00FF0036
:10429000FF00FF00FF00FF00FF00FF00FF00FF0026
:1042A000FF00FF00FF00FF00FF00FF00FF00FF0016
:1042B000FF00FF00FF00FF00FF00FF00FF00FF0006
:1042C000FF00FF00FF00FF00FF00FF00FF00FF00F6
:1042D000FF00FF00FF00FF00FF00FF00FF00FF00E6
:1042E000FF00FF00FF00FF00FF00FF00FF00FF00D6
:1042F000FF00FF00FF00FF00FF00FF00FF00AA001B
:00000001FF
